:100000000C943D050C9484050C9484050C94840593
:100010000C9484050C9484050C9484050C9484053C
:100020000C9484050C9484050C9406230C94D8231A
:100030000C94D9190C9484050C9484050C948405B3
:100040000C9484050C9484050C9484050C9484050C
:100050000C9484050C94261A0C9484050C94840545
:100060000C9484050C9484050C9484050C948405EC
:100070000C9484050C9484050C9484050C948405DC
:100080000C9484050C9484050C9484050C948405CC
:100090000C9484050C9484050C9484050C948405BC
:1000A0000C9484050C9484050C948405120F120F93
:1000B000440F440F910FAF0F07110711F10F861076
:1000C00097109710F710071107110011A711A7112A
:1000D000B911B911B011B911B911B911A711A711FD
:1000E000B511B911B911B51145246C2464256C24DE
:1000F0006425B824DB24642532254125165C1E00C6
:100100001F002000210022002300240025002600DB
:1001100027002A002B0014001A0008001500170001
:100120001C0018000C00120013004C0039000400E1
:100130001600070009000A000B000D000E000F005A
:1001400033003400E1001D001B000600190005000B
:1001500011001000360037003800D95CE0000B5D5C
:10016000E300E200095D2C002C000A5D5000510004
:1001700052004F0035021E021F02200221022202FD
:10018000230224022502260227022A0035021E022B
:100190001F0220022102220223022402250226023B
:1001A00027024C004C003A003B003C003D003E0062
:1001B0003F002D022E022F023002310201004000CA
:1001C00041004200430044004500010046004A004F
:1001D0004D000100010001000100010001000100CB
:1001E00001000100AC00AE00A800AB0035001E000D
:1001F0001F002000210022002300240025002600EB
:1002000027002A0035001E001F00200021002200C8
:10021000230024002500260027004C004C003A0053
:100220003B003C003D003E003F002D002E002F0013
:100230003000310001004000410042004300440012
:100240004500010049004B004E0001000100010083
:10025000010001000100010001000100AC00AE003E
:10026000A800AB000000000000000000000000003B
:10027000000000000000000000000000000000007E
:10028000000000000000000000000000000000006E
:10029000000000000000000000000000000000005E
:1002A000000000000000000000000000000000004E
:100870000000000000000000000000003A003B0003
:100880003C003D003E003F0040004100420043006C
:10089000440045000100005C010001000100145CFF
:1008A0000100010001000100010001000100010040
:1008B0000100010001000100010001000100010030
:1008C0000100010001000100010001000100010020
:1008D0000100010001000100010001000100010010
:1008E0000100010001000100010001000100010000
:1008F00001000100040330000000240348006100EF
:100900006E006400770069007200650064002000DA
:100910005000720065006F006E0069006300000007
:100920000A034E00650069006C000000040309041E
:1009300009023B00020100A0FA09040000010301C2
:10094000010009211101000122400007058103086F
:10095000000A09040100010300000009211101003F
:100960000122BC000705820320000A1201100100C9
:10097000000008EDFE6160010001020301050109AC
:1009800002A10185020901A1000509190129051526
:100990000025019505750181029501750381010509
:1009A00001093009311581257F95027508810609F5
:1009B000381581257F950175088106050C0A3802D6
:1009C0001581257F950175088106C0C00501098044
:1009D000A101850319012AB700150126B700950169
:1009E00075108100C0050C0901A101850419012AB7
:1009F000A002150126A002950175108100C0050115
:100A00000906A1018505050719E029E7150025015B
:100A10009508750181020507190029EF15002501C8
:100A200095F07501810205081901290595057501E3
:100A30009102950175039101C005010906A1010507
:100A40000719E029E7150025019508750181029530
:100A500001750881010507190029FF150026FF000F
:100A60009506750881000508190129059505750188
:100A70009102950175039101C00011241FBECFEFB3
:100A8000DAE0DEBFCDBF04B603FE27C080918A0244
:100A900090918B02A0918C02B0918D028730904B87
:100AA000A740B04BD1F410928A0210928B021092A0
:100AB0008C0210928D0214BE84B7877F84BF0FB65C
:100AC000F894A895809160008861809360001092EE
:100AD00060000FBEE0E0F8E3099511E0A0E0B1E0AE
:100AE000E4E1FCE402C005900D92A838B107D9F703
:100AF00022E0A8E8B1E001C01D92AA38B207E1F7F0
:100B00000E9435200C9408260C940000CF93DF93AC
:100B1000EC010E942A18BE0180E090E0DF91CF91A5
:100B20000C948B15CF93FB0189302DE59207A9F02A
:100B300020F488309D4549F032C08A302DE5920777
:100B400079F08B309D4501F12AC0C281CC2341F15F
:100B500081E090E00E9486051DC0C28181E002C054
:100B6000C28182E0CC2341F00E94EB1540E162E0BB
:100B700081E00E9475060EC00E940C1640E162E002
:100B800081E00E9475060CC0C28180E1CC2321F077
:100B90000E94EB15C0E004C00E940C1601C0C1E029
:100BA0008C2FCF91089581E008950C9492050895BB
:100BB0000C94D7051F93CF93DF9300D000D01F92E2
:100BC000CDB7DEB749835A836B833091A001898109
:100BD0009A81311114C0662359F0222349F00E94F2
:100BE000E016182F682F89819A810E94891603C008
:100BF0000E94B416182F69817A81812F04C00E9447
:100C0000E01669817A810F900F900F900F900F90EE
:100C1000DF91CF911F910C94F206FC01262F4081A9
:100C200051816281738184810C94DA05CF93DF93C3
:100C3000EC0160E00E940D06BE01DF91CF910C94A3
:100C4000D8058F929F92AF92BF92CF92DF92EF9290
:100C5000FF920F931F936B017C0181E090E0A0E075
:100C6000B0E04C015D0104C0880C991CAA1CBB1C9F
:100C70004A95D2F7AC01BD0104C0440F551F661F51
:100C8000771F2A95D2F7482959296A297B2904C058
:100C9000880F991FAA1FBB1F0A95D2F78A019B01D3
:100CA0000C211D212E213F21401751076207730798
:100CB00039F4BC01CD016C297D298E299F290AC0F8
:100CC00080959095A095B095BC01CD016C217D21BA
:100CD0008E219F211F910F91FF90EF90DF90CF9079
:100CE000BF90AF909F908F9008950F93382F262F2D
:100CF00060910102709102028091030290910402BE
:100D0000042F432F0E9421060F910C94C5150E94B9
:100D10001218811102C00E94BC180C9411090C9485
:100D20000D0908950C94910681E008950C949406A1
:100D3000CF93C82F0E9492068C2F0E949606CF91C7
:100D4000089508950E9495110E94A1062FEF84E353
:100D50009CE0215080409040E1F700C000000C94DE
:100D60004C1A0F931F93CF93DF93EC0161E00E9425
:100D70000D068C01BE010E94D505882349F1BE01F4
:100D8000C8010E94A10A882319F1BE01C8010E946E
:100D9000E20A8823E9F0BE01C8010E940D0C8823F5
:100DA000B9F08A81882369F001158CE5180731F0C4
:100DB0000E3D1C4531F40E94BC180AC00E94A206D8
:100DC00007C0CE01DF91CF911F910F910C94D305F5
:100DD00080E0DF91CF911F910F91089580E090E026
:100DE000089508952CE3829FC0011124FC012CE09A
:100DF000729FE00DF11D1124E60FF11DEE0FFF1F94
:100E0000E450FF4F859194910895880F991FFC013C
:100E1000EC50F74F859194910895CF93DF930E9402
:100E2000F2060E942508EC018115904508F041C0AA
:100E3000C11580E4D80708F0D1C0C83ED10510F52F
:100E4000C03ED10508F0FDC0C83AD10578F4C53AD6
:100E5000D10508F0A2C0C130D10509F4F2C008F4F0
:100E6000EEC0C430D10508F0ECC0E9C0CF3BD105DD
:100E700008F49BC0C03CD10508F4E1C0CE01805C01
:100E800091099EC0C11590E2D90758F4C11521E01F
:100E9000D20708F0D6C0C03FD10508F4D0C0D06555
:100EA000D0C0C11580E3D80708F08EC0CE019F7076
:100EB00087C0C11595E5D90708F043C0C11524E5E1
:100EC000D20708F0A2C0C11582E5D80708F5C11500
:100ED00091E5D90708F085C0CE0174E09695879515
:100EE0007A95E1F783709C2F937021E030E002C087
:100EF000220F331F9A95E2F73C68382BCF70C695C6
:100F0000C69580E2C89FE0011124C22BD32B99C063
:100F10009E01237033278C2F86958695C115D34566
:100F200008F064C0C1E0D0E002C0CC0FDD1F2A95FC
:100F3000E2F720E2829FC0011124C82BD92BDC6884
:100F400080C0C11529E5D207A0F4C11588E5D807EE
:100F500008F060C0C11596E5D90708F070C08C2F65
:100F60000E94B9088F71C82FD0E0DC2FCC27D06247
:100F700068C0C1152AE5D20708F451C0CE019056C9
:100F80008115904208F05BC08D2F8F710E94B908C7
:100F9000DD27D0628F71D82B54C0C55AD0E0CD5B0D
:100FA000DE4FC881D0E0D0644CC0C85AD0E0CC0F2E
:100FB000DD1FCB5EDE4F0990D881C02DD46441C0C7
:100FC0000E940507EC013DC0CE019927D3FF03C065
:100FD000EC01D86C36C0EC01D06C33C0DF70D06A45
:100FE00030C0DC2FCC27C16FD06A2BC0C1E0D0E06D
:100FF00002C0CC0FDD1F2A95E2F720E2829FC001DC
:101000001124C82BD92BDA681CC0DC2FCC27C46F65
:10101000D06A17C0DC2FCC27C06FD06A12C08C2FCB
:101020008F700E94B90894E0D695C7959A95E1F71C
:10103000CF70D0E0DC2FCC27D069C82B02C0C0E035
:10104000D0E0CE01DF91CF9108958238910569F10A
:10105000B0F48133910509F46DC048F489329105EB
:1010600009F463C08A32910509F469C00895853393
:10107000910509F455C089339105B9F00895833E6F
:10108000910569F138F4803E9105B1F0823E9105F9
:1010900009F10895863E9105A9F1873E9105B9F1C0
:1010A000843E910509F064C023C020917B0220FD9D
:1010B0004FC021FD4DC0089580917B0280FD44C04A
:1010C00080917C0280FF44C080917B0284FD42C0FD
:1010D00083EE4DC080917B0282FF38C0F5CF8091B6
:1010E0007B0282FD33C080917C0280FD31C0ECCF59
:1010F00080917C0281FF32C080917B0284FD2AC0F6
:1011000087EE35C080917B0283FF26C0F5CF8091AA
:101110007B0283FD21C080917C0281FD1FC0ECCF4A
:1011200080917B0285FD1CC01DC080917B0285FDE6
:1011300019C016C080917B0286FD16C017C0809131
:101140007B0286FD13C010C089E311C082EE0FC080
:1011500080EE0DC080E00BC086EE09C084EE07C0B3
:1011600089E205C085E303C08AE201C081E390E023
:10117000089590917B0292FF0DC0282F287128308E
:1011800019F4877F846006C0282F2471243011F45D
:101190008B7F886093FF0DC0282F2871283119F4A8
:1011A000877E846106C0282F2471243111F48B7E40
:1011B000886120917C0220FF0DC0382F38713830B3
:1011C00019F4877F816006C0382F3171313011F4F6
:1011D0008E7F886021FF0DC0282F2871283119F4D7
:1011E000877E816106C0282F2171213111F48E7E06
:1011F000886194FD877E0895E82FF0E0EE0FFF1FD1
:10120000E559FD4F808191810895089580EA8A957E
:10121000F1F7089508950C940A090C940B090C94A5
:101220000A090C940F09CF93DF93A2E5B1E047E5DB
:1012300051E061E070E08D91E82FE295EF70F0E011
:1012400021A18F70EB0102C0CC0FDD1F8A95E2F760
:10125000CE019C2F9095922391A392A1892B82A3DA
:101260004A175B0741F7A6E4B1E042E551E061E0CF
:1012700070E08D91E82FE295EF70F0E021A18F7082
:10128000EB0102C0CC0FDD1F8A95E2F7CE019C2F47
:101290009095922391A392A1892B82A34A175B0771
:1012A00041F7E1E6F2E0ABE6B2E08BE692E01192C4
:1012B00011921D921D928E179F07C9F785E00E941B
:1012C000F209DF91CF910C9487066F927F928F92F3
:1012D0009F92AF92BF92CF92DF92EF92FF920F93C5
:1012E0001F93CF93DF9382E5C82E81E0D82E01E6CD
:1012F00012E09BE6A92E92E0B92E712C88248394EB
:10130000912CF60181916F01C82FC295CF70D0E06A
:1013100099A18F70740101C0EE0C8A95EAF7892FAC
:101320008E2989A38AA16E2C609486218AA30E94AB
:101330000609E6E4F1E040E050E020E030E06191B1
:10134000A62FA295AF70B0E090968C9190E06F7050
:1013500002C0959587956A95E2F780FD08C0C401A3
:10136000042E02C0880F991F0A94E2F702C080E0A1
:1013700090E0282B392B4F5F5F4F4C305105F9F629
:1013800089A1682269A28AA1E82AEAA2F8018081DB
:1013900091812817390721F03183208381E001C032
:1013A00080E0782A0E5F1F4FA016B10609F0A9CF82
:1013B000272D45E06BE672E081E692E00E94F3099A
:1013C0000E948F06872DDF91CF911F910F91FF9083
:1013D000EF90DF90CF90BF90AF909F908F907F90D5
:1013E0006F9008950895FF920F931F93CF93DF930B
:1013F000F82E092F162FD72FC42F222349F081E072
:1014000080938A010E940B1A90938901809388012E
:1014100080918A018823D9F0809188019091890177
:101420000E94171A069798F0EF2DF02FA12FBD2FCD
:1014300080E090E04C2F50E08417950734F4219120
:1014400031912D933D930196F7CF10928A01DF9150
:10145000CF911F910F91FF9008950F931F93CF93FA
:10146000DF93C62FD42F122FFC0182818823C9F06D
:1014700060938D010E940B1A90938C0180938B01D5
:1014800080E28C0F883008F057C0C77081E001C03F
:10149000880FCA95EAF7DF91CF911F910F910C94B5
:1014A000CE0E80918D01681330C080918B01909198
:1014B0008C010E94171A883C910538F500E20D0F47
:1014C000CD17B9F080E28C0F883040F4C77081E00E
:1014D00001C0880FCA95EAF70E94D50E083028F59A
:1014E00081E09D2F977001C0880F9A95EAF70E94BE
:1014F000CE0E812F0E94BB0E0830F0F4D77081E031
:1015000001C0880FDA95EAF70AC080E28C0F8830B4
:1015100098F4C77081E001C0880FCA95EAF7DF919F
:10152000CF911F910F910C94D50E812FDF91CF9108
:101530001F910F910C94BB0EDF91CF911F910F91D2
:1015400008959C01CB01233F4CE53407F9F078F472
:10155000283DFCE53F07B9F0293D4CE5340711F182
:10156000273D3C4531F526E241EE61EE1EC0253FA8
:10157000FCE53F0799F070F0263F3C45D1F427E2A7
:1015800045EE66EE12C027E245EE0EC026E241EEC1
:1015900060EE0BC027E245EE64EE07C026E241EEA6
:1015A00062EE03C028E241E065EE0E942D0A80E071
:1015B0000895FC018281882319F010928D0108950D
:1015C00081E00895CF93DF93EC01FB0182818823B2
:1015D00009F41FC1C230FCE5DF0708F41BC1C631A6
:1015E0009CE5D90738F09E012A5F3C45293031053A
:1015F00008F010C10E942F1890937C0280937B0208
:10160000C031ECE5DE0709F4C3C008F041C0C830C2
:101610008CE5D80709F49AC0F0F4C430ECE5DE0795
:1016200009F487C068F4C2308CE5D80709F477C0A4
:10163000C330DC4509F0E3C080917B02826076C054
:10164000C630ECE5DE0709F46EC008F07BC080917F
:101650007B0288606BC0CC308CE5D80709F485C06C
:1016600068F4CA30ECE5DE0709F474C008F079C00C
:101670000E94951180917B02806858C0CE308CE525
:10168000D80709F476C008F07FC080917B028BC038
:10169000CB3FECE5DE0709F44FC018F5C3318CE50C
:1016A000D80709F47DC078F4C131ECE5DE0709F410
:1016B00073C0C231DC4509F0A2C00E94951180912F
:1016C0007B028F7733C0C5318CE5D80709F472C02F
:1016D00008F486C0CA3FDC4509F091C080917C02C5
:1016E0003EC0CF3FFCE5DF0709F45FC058F4CD3FB3
:1016F0009CE5D90709F444C008F43FC080917C02FE
:1017000082602DC0C130FDE5DF0709F475C008F423
:101710005DC0C230DD4509F072C080E06EC08091CE
:101720007B02816003C080917B02806180937B0299
:1017300066C080917B0211C080917C0282608093A0
:101740007C025DC080917B028062F0CF80917B0241
:101750008064ECCF80917B0288608460E7CF8160F9
:10176000EECF80917B028E7FE1CF80917B028D7FD7
:10177000DDCF80917B02877FD9CF80917C0218C01A
:1017800080917C028D7FDBCF80917B028F7ECECFDC
:1017900080917B028F7DCACF80917B028F7BC6CFE9
:1017A00080917B02877F8B7FC1CF80917C028D7F70
:1017B0008E7FC5CF80917B0282FB222720F991E0AA
:1017C000922790FB82F990FB83F9B0CF80917C0245
:1017D000982F909591708E7F892B90FB81F9AFCFD8
:1017E0000E94951180917B0287FB222720F991E0CE
:1017F000922790FB87F99ACF81E00E94BE188091D2
:101800007B0290917C020E9440180E94951180E01A
:1018100001C081E0DF91CF910895CF93DF938631AE
:101820009C4541F5EB010E946117982F8A81209118
:10183000000130910101882379F09A7A81E009F45E
:1018400080E080938E01911102C069E201C065E3DE
:10185000C9010E9459190AC080918E01811102C0EC
:1018600069E201C065E3C9010E9464190E94AF17D3
:1018700080E001C081E0DF91CF91089590939401C1
:10188000809393010895E0919301F0919401309732
:1018900021F00190F081E02D099480E00895E0911D
:1018A0009301F0919401309799F020911401222333
:1018B00059F020917B0227FF07C0DC012C91119683
:1018C0002C93119725E02C930280F381E02D09944D
:1018D0000895E0919301F0919401309739F022E05E
:1018E000DC012C930480F581E02D0994089520916A
:1018F0009101309192012817390771F0909392016C
:1019000080939101E0919301F0919401309721F03F
:101910000680F781E02D0994089520918F01309180
:1019200090012817390771F09093900180938F01EF
:10193000E0919301F0919401309721F00084F185BA
:10194000E02D0994089585B7806885BF85B78068C4
:1019500085BF089508950C94AA0C0C94AB0C0C94BC
:10196000AA0C0C94AA0C0E94A30C0E94AF0C0C941D
:10197000AD0C81E008950C94B90C0E94021A0E94EB
:1019800013090E94BC1A0C94B10C7F928F929F9203
:10199000AF92BF92CF92DF92EF92FF920F931F937D
:1019A000CF93DF93CDB7DEB72A970FB6F894DEBF9B
:1019B0000FBECDBF0E9465090E94BB0C811111C0F2
:1019C0008FEF89838A831B820E940B1A8160782F94
:1019D0009D838C8349815A816B818D810E94750D15
:1019E0004FC046E9A42E41E0B42E00E010E0702E76
:1019F000802F0E94FC086C01F501819091905F019D
:101A0000882699268114910431F40F5F1F4F053009
:101A1000110569F7D5CF80912E0281FD0E9405093D
:101A200080E0EE24E394F12C94012E213F21232B1E
:101A300009F18E837F82CE20DF2081E0CD2809F45A
:101A400080E088870E940B1A8160782F9A878987A7
:101A50004E815F8168858A850E94750D000F111F78
:101A6000F801EA56FE4F80819181E826F926F1823D
:101A7000E08206C08F5FEE0CFF1C8C30A9F6C5CF4C
:101A80000E94701D0E94430C909195018917C9F026
:101A90000E94430C809395012A960FB6F894DEBFFE
:101AA0000FBECDBFDF91CF911F910F91FF90EF90AF
:101AB000DF90CF90BF90AF909F908F907F900C94CD
:101AC00098062A960FB6F894DEBF0FBECDBFDF9101
:101AD000CF911F910F91FF90EF90DF90CF90BF902B
:101AE000AF909F908F907F900895CF93DF93CDB765
:101AF000DEB72B970FB6F894DEBF0FBECDBF4F8376
:101B0000588769877A878B87DE01119686E0FD0109
:101B100011928A95E9F785E0FE01379601900D92C2
:101B20008A95E1F749815A816B817C818D819E8103
:101B30000E944E142B960FB6F894DEBF0FBECDBF99
:101B4000DF91CF910895FC01808191810E9422173D
:101B50000895CF93882309F4A4C0C82F8238C1F414
:101B60000E94430C81FD9DC069E38091000190912A
:101B700001010E9459190E94AF172FEF81EE94E0E6
:101B8000215080409040E1F700C0000069E319C097
:101B9000833801F50E94430C80FD83C063E580918A
:101BA0000001909101010E9459190E94AF172FEF77
:101BB00081EE94E0215080409040E1F700C00000A9
:101BC00063E580910001909101010E946419CF9119
:101BD0000C94AF178438C1F40E94430C82FD61C09D
:101BE00067E480910001909101010E9459190E94BF
:101BF000AF172FEF81EE94E0215080409040E1F745
:101C000000C0000067E4DDCF8CEF8C0F813AD0F488
:101C10006C2F80910001909101010E94D9188823B6
:101C200049F06C2F80910001909101010E9464198C
:101C30000E94AF176C2F80910001909101010E94CA
:101C40005919C5CF80E28C0F883048F4C77081E005
:101C500001C0880FCA95EAF70E946417B8CFEBE578
:101C6000EC0FE33040F4F0E0EB57FE4F808190E062
:101C7000CF910C94770CE8E5EC0FE73150F4F0E0ED
:101C8000EE0FFF1FE95AFE4F80819181CF910C9496
:101C90008D0CC03F30F08C2F0E94781CCF910C949B
:101CA000651DCF910895882309F464C0823879F4C2
:101CB0000E94430C81FF5EC069E380910001909116
:101CC00001010E9459190E94AF1769E310C08338BF
:101CD000B1F40E94430C80FF4DC063E58091000188
:101CE000909101010E9459190E94AF1763E58091FC
:101CF0000001909101010E9464190C94AF1784387F
:101D000079F40E94430C82FF35C067E480910001A2
:101D1000909101010E9459190E94AF1767E4E7CF23
:101D20009CEF980F913A10F4682FE1CF90E2980F52
:101D3000983050F4877091E001C0990F8A95EAF7C6
:101D4000892F0E946A17D9CF9BE5980F933020F412
:101D500080E090E00C94770C98E5980F973120F490
:101D600080E090E00C948D0C803F20F00E94E01CFD
:101D70000C94651D0895CF93C82F0E94A90DC933F7
:101D800049F42FEF87EE93E0215080409040E1F737
:101D900000C000008C2FCF910C94530E882321F0AB
:101DA0000E9464170C94AF170895882321F00E94B5
:101DB0006A170C94AF170895CF92DF92EF92FF92BB
:101DC0000F931F93CF93DF937C01062FC72FFC0146
:101DD000158112951F70D281D1110E9481170E9426
:101DE0005A17882399F0DD2389F08C2F807F803467
:101DF00021F080E2800F883048F082E00E94F917DD
:101E00000E945A1791E0D82ED92601C0D12CCC2E91
:101E1000C2948FE0C8228C2D90E0FC01EA5AFF4F5B
:101E20000C94AC258C2F807FCF70882311F0C29545
:101E3000C07FDD2399F0CC2309F4C4C180E2800F78
:101E4000883010F0011104C08C2F0E94641703C069
:101E50008C2F0E9474170E94AF17B4C1802F0E946C
:101E6000530ECC2309F4D3C180E2800F883010F0E8
:101E7000011104C08C2F0E946A1703C08C2F0E948E
:101E80007A170E94AF17C3C18C2F807FCF7080322A
:101E900011F0C295C07F002319F00130C9F022C0B3
:101EA000DD2371F0112341F0113031F40E949417B9
:101EB0008C2B0E949C17ABC10E9494178C2B1DC0C9
:101EC000112319F0113009F4A2C10E94A51725C0F1
:101ED000DD2321F0163008F09AC10EC0153008F04D
:101EE00096C11BC0DD2361F0112331F0F70185811C
:101EF00080FF68C18F7085838C2F0E94CE0E87C1B2
:101F0000112359F0093309F06EC1FFEF27EE83E08A
:101F1000F15020408040E1F764C18C2F0E94D50E23
:101F200076C18C2F86958695837019F0813061F08B
:101F30006EC1DD2321F0802F9C2F937002C080E0C2
:101F400090E00E94770C6BC1DD2321F0802F9C2F45
:101F5000937002C080E090E00E948D0C60C1DD2390
:101F6000F9F0053F51F0063F71F0043FA9F480916C
:101F700075029091760281600BC0809175029091FC
:101F80007602826005C0809175029091760284602D
:101F90009093760280937502802F0E94781C1EC059
:101FA000053F51F0063F71F0043FA9F4809175029E
:101FB000909176028E7F0BC080917502909176028F
:101FC0008D7F05C080917502909176028B7F9093F2
:101FD000760280937502802F0E94E01C0E94651D8E
:101FE0001EC18C2F837009F045C0D11114C1402F40
:101FF000429546954770440F440F602F6F70862FAF
:1020000090E0A0E0B0E0042E04C0880F991FAA1F42
:10201000BB1F0A94D2F704FF10C00FE010E020E0CD
:1020200030E004C0000F111F221F331F4A95D2F762
:10203000009510952095309503C000E010E09801C0
:10204000C695C695C370BC01CD01602B712B822B48
:10205000932BC23049F058F4C13019F00E949F15FB
:10206000DAC00E948D15D7C00E94B115D4C00E945D
:102070008B15D1C0DD2319F08C2F817001C086959E
:10208000882309F4C8C0402F429546954770440FF5
:10209000440F602F6F70862F90E0A0E0B0E0042E18
:1020A00004C0880F991FAA1FBB1F0A94D2F704FF10
:1020B00010C00FE010E020E030E004C0000F111F5E
:1020C000221F331F4A95D2F7009510952095309521
:1020D00003C000E010E09801C695C695C370BC012E
:1020E000CD01602B712B822B932BC23049F058F419
:1020F000C13019F00E9464168EC00E9452168BC027
:102100000E94761688C00E94C51585C0CF70DD2359
:1021100039F08C2F0E94EB15802F0E94CE0E7BC0D1
:10212000802F0E94D50E8C2F0E940C1674C0023F87
:1021300001F128F4003F41F0013FA1F03FC0033F0F
:10214000F9F0043F39F13AC0DD2341F0153008F0D1
:102150005EC08C2F8F710E94311659C0163008F066
:1021600056C0F7CFDD2339F08C2F8F710E94EB150D
:102170004EC0DD23C9F38C2F8F710E940C1647C00F
:10218000DD2329F08C2F8F710E94D61540C00E944C
:10219000D1153DC0DD2349F0CF718C2F0E94EB1586
:1021A00063E08C2F0E94E41732C081E00E94F9178F
:1021B000123068F182E00E94F91729C0DD2331F066
:1021C000112391F2802F0E94A90D21C0112399F2B1
:1021D000093349F49FEFE7EEF3E09150E040F0401F
:1021E000E1F700C00000802F0E94530E10C04C2F5A
:1021F0004F70602FC7010E94EE060E94FC140FC0B2
:102200004C2F4F70602FC7010E94F10608C088EF65
:102210008C0D843020F40E94430C0E949806DD202F
:10222000C9F00E94561780FD15C0F70112820E9466
:1022300050170E94EB15C7010E944B110E945017C6
:10224000DF91CF911F910F91FF90EF90DF90CF9092
:102250000C940C16DF91CF911F910F91FF90EF908E
:10226000DF90CF9008950F931F93CF93DF93EC01EE
:10227000688179818A810E942D178C010E948816BD
:102280000E947915B801CE010E94DC0EDF91CF913A
:102290001F910F910895CF93DF93EC01988189816D
:1022A0002B813C81232B31F08F3F31F481E09F3F24
:1022B00019F403C081E001C080E080FD19C0CE01A7
:1022C0000E94B10681110CC00E945A17882381F028
:1022D0008A81882369F082E0DF91CF910C94F9170D
:1022E000CE010E943311CE01DF91CF910C941606DE
:1022F000DF91CF9108950E9481170E9491170E944B
:10230000AF170E948F1E0E94651D80E090E00E9422
:10231000770C80E090E00C948D0C809100019091FE
:1023200001010E946F190C947B110E9471170C948B
:102330008D11E92FE295EF704E2F50E0FA013297A0
:10234000EE30F105B0F4EA59FF4F0C94AC25803F14
:1023500091F018F4883E68F40EC0843F51F40BC02D
:10236000883E48F0813F29F406C093FB882780F916
:10237000089580E0089581E008950E9422170E9448
:1023800099110895CF93DF9300D000D01F92CDB75D
:10239000DEB70F900F900F900F900F90DF91CF91BD
:1023A0000895CF93DF9300D000D000D0CDB7DEB733
:1023B00026960FB6F894DEBF0FBECDBFDF91CF914A
:1023C00008951F93CF93DF93C091A10116E08091F0
:1023D000A201C81799F0D0E01C9FF0011D9FF00DDD
:1023E0001124ED55FE4F40815181628173818481BA
:1023F00095810E94D1112196C770E9CFDF91CF91CD
:102400001F9108954091D3015091D4016091D5015D
:102410007091D6018091D7019091D8010C94D1117F
:102420000F931F93CF93DF938091D80182958F7084
:1024300009F05DC08091D501882309F458C08091CE
:10244000A1011091A2016091D3017091D401C091BA
:10245000D601D091D70191E06F3F09F090E0292F8C
:1024600006E0811709F443C0209721F07F3F21F057
:1024700030E003C031E001C0322F90E030FD34C0C5
:10248000089FF001099FF00D1124DF01AD55BE4FEB
:1024900011963C911197371327C03C91361324C0F5
:1024A00012963C91129731111FC013964D915C9179
:1024B00014974C1B5D0B483C5105B0F48091D8013A
:1024C0008F7080618093D801E855FE4F80818F70B6
:1024D0008061808383ED91E00E944B11DF91CF9169
:1024E0001F910F910C94E11101968770BACFDF9183
:1024F000CF911F910F9108959F92AF92BF92CF926B
:10250000DF92EF92FF920F931F93CF93DF93CDB79C
:10251000DEB761970FB6F894DEBF0FBECDBF8C015A
:1025200085E0F801DE011D9601900D928A95E1F794
:10253000F80140815181E2809091D3016091D401F2
:102540002091D6013091D7012115310531F06F3F2F
:1025500031F481E09F3F19F403C081E001C080E0C5
:10256000F82FF1709F2E80FD46C1F801A380B48042
:1025700083EDC82E81E0D82EF090D501F501E21B45
:10258000F30BFF2009F4DFC08091D801E83CF1058E
:1025900008F09BC0282F207F09F052C0561313C0AB
:1025A000491311C0FE2CE1100EC08F708061809322
:1025B000D8010E940212C6010E944B118091D801DD
:1025C000F801858358C1AB2831F05F3F31F481E0D9
:1025D0004F3F19F403C081E001C080E080FD03C0DB
:1025E00081E08E2502C080E090E0F82FF170FF2E90
:1025F00080FF1CC08091A1012091A20136E08217CA
:1026000009F417C190E0389FF001399FF00D1124B3
:10261000ED55FE4F6181561306C06081461303C01D
:102620006281E61203C001968770E9CFFE2CEE208E
:1026300009F421C18091D80181608093D8015AC0EA
:10264000561306C0491304C0E11002C0F8019FC030
:102650004D875E878D859E850E94BD11882379F107
:10266000EE2069F12091D801822F82958F7090E041
:10267000029774F08091D3019091D40198878F8351
:102680001986BB86AA862C87CE0107960E944B111D
:1026900086E0F801A3EDB1E001900D928A95E1F793
:1026A0000E9410120E9402120DC0561729F14D8788
:1026B0005E878D859E850E94BD1181112CC0C80149
:1026C0000E944B11FF24F394D6C0282F207F69F776
:1026D0007A2DB98AA88A6E2D89890E94C21183ED4C
:1026E00091E00E944B1186E0F60111928A95E9F77C
:1026F0000E940212F12CBFC04913D9CFE110D7CFED
:10270000F8018583C8010E944B1186E0F601119201
:102710008A95E9F7B0C0EE2091F22091D801822F7E
:1027200082958F7090E002970CF4B2CF8091D30124
:102730009091D4019A8389831B82BD82AC822E83BF
:10274000CE010196A3CFE83CF10508F047C0FE2C6E
:10275000EE2009F4B4CF561330C049132EC0209197
:10276000D80120FD21C0822F82958F70482F50E024
:1027700041155105C9F0F80125834F30510541F04D
:102780008F5F982F9295907F822F8F70892B8583F2
:10279000C8010E944B1186E0F801A3EDB1E0019061
:1027A0000D928A95E1F742C086E0F801A3EDB1E011
:1027B00001900D928A95E1F75EC04D875E878D8509
:1027C0009E850E94BD11811163CF8091D8018160E7
:1027D0008093D801C8010E944B114DC07A2DB98A4F
:1027E000A88A6E2D89890E94C21186E0F601119295
:1027F0008A95E9F71BC0EE2009F461CF4D875E870B
:102800008D859E850E94BD11F82E882309F457CF2F
:1028100086E0F801A3EDB1E001900D928A95E1F711
:1028200083ED91E00E94A30D0E9410120E940212FB
:1028300022C04D875E878D859E850E942217292F95
:1028400022952F70223028F49F7039F0811105C035
:102850000BC0243028F49F7049F4805E883020F04B
:10286000C8010E944B119F2CF92C05C0F8019581DD
:10287000907F99F7F9CF8F2D61960FB6F894DEBF50
:102880000FBECDBFDF91CF911F910F91FF90EF90C1
:10289000DF90CF90BF90AF909F9008951F93CF93FC
:1028A000DF93CDB7DEB72C970FB6F894DEBF0FBE1F
:1028B000CDBF4F83588769877A878B879C87CE01E6
:1028C00007960E947C128823D1F09F8188852A85F3
:1028D0003B85232B31F08F3F31F481E09F3F19F48A
:1028E00003C081E001C080E080FD47C04F81588572
:1028F00069857A858B859C850E94D1113EC086E0D2
:10290000FE013796DE01119601900D928A95E1F74E
:10291000FF81E8856A857B856115710531F0EF3FA0
:1029200031F481E0FF3F19F403C081E001C080E091
:1029300080FD23C02091A20130E0C901019687707B
:1029400099274091A10150E084179507F1F1F9838F
:10295000EA837D836C8396E0929FD001939FB00DB4
:102960001124AD55BE4FFE01319601900D929A95FE
:10297000E1F78093A2010E94E11116E08091A1018C
:102980009091A201891771F1189FC00111248D55F2
:102990009E4F0E947C12882329F1E091A1011E9F85
:1029A000F0011124ED55FE4F408151816281738108
:1029B000848195810E94D1118091A10190E00196BE
:1029C000877099278093A101D9CF0E949511109209
:1029D000A2011092A101E3EDF1E086E0DF011D927A
:1029E0008A95E9F72C960FB6F894DEBF0FBECDBFDF
:1029F000DF91CF911F910895EF92FF920F931F9354
:102A0000CF93DF938C01892B09F46CC0F12CEE2459
:102A1000E394E8012196F8018491843740F48430EE
:102A200008F051C0813081F0823019F15BC08537E8
:102A300009F444C0A8F19CE7980F903708F052C001
:102A40008F770E94530E41C00E5F1F4FFE0184918D
:102A500090E2980F983050F48770FE2D01C0FF0F60
:102A60008A95EAF78F2F0E94841714C00E94A90D3F
:102A70002DC00E5F1F4FFE01849190E2980F983099
:102A800060F48770FE2D01C0FF0F8A95EAF78F2F43
:102A90000E948A170E94AF1719C00E94530E16C0D9
:102AA0000E5F1F4FFE01C491CC2381F08FE99FE0A0
:102AB0000197F1F700C00000C150F6CF0E5F1F4F25
:102AC000FE01F49003C00E94A90D8E018F2D882372
:102AD00009F49FCFEFE9FFE03197F1F700C0000064
:102AE0008150F5CFDF91CF911F910F91FF90EF9023
:102AF0000895089508950C947A150C947B150E94FE
:102B00007D156093050270930602809307029093EF
:102B100008020C947B110C947F150F931F93009166
:102B20000502109106022091070230910802602BE5
:102B3000712B822B932B1F910F910C947F150F9368
:102B40001F93009105021091060220910702309117
:102B5000080260237123822393231F910F910C9409
:102B60007F150F931F93009105021091060220918B
:102B700007023091080260277127822793271F914F
:102B80000F910C947F150C947A150E94C3156093D5
:102B900001027093020280930302909304020C944A
:102BA0007B1160E070E0CB010C94C5150F931F936F
:102BB00041E050E060E070E08A019B0104C0000F3A
:102BC000111F221F331F8A95D2F7C901B8011F9127
:102BD0000F910C94C5150F931F9341E050E060E0F6
:102BE00070E004C0440F551F661F771F8A95D2F707
:102BF0008091010290910202A0910302B09104021F
:102C00008A019B01082B192B2A2B3B2BC901B801E8
:102C10001F910F910C94C5150F931F9341E050E045
:102C200060E070E004C0440F551F661F771F8A954F
:102C3000D2F74095509560957095809101029091E2
:102C40000202A0910302B09104028A019B010823B1
:102C500019232A233B23C901B8011F910F910C941A
:102C6000C5150F931F9341E050E060E070E004C091
:102C7000440F551F661F771F8A95D2F78091010276
:102C800090910202A0910302B09104028A019B017B
:102C9000082719272A273B27C901B8011F910F913F
:102CA0000C94C5150F931F9300910102109102021D
:102CB0002091030230910402602B712B822B932B05
:102CC0001F910F910C94C5150F931F930091010252
:102CD00010910202209103023091040260237123BB
:102CE000822393231F910F910C94C5150F931F936B
:102CF000009101021091020220910302309104021E
:102D000060277127822793271F910F910C94C51577
:102D100008952CE0929F800D1124E82FE695E6950A
:102D2000E695877051E001C0550F8A95EAF785E076
:102D3000E89FF0011124E752FE4F20E030E070E000
:102D40004081CB01022E02C0969587950A94E2F746
:102D50008170819584278523842781932F5F3F4F3E
:102D60002530310569F708952CE0929F800D1124DC
:102D7000682F669566956695982F977085E0689F91
:102D8000B001112440E050E080E0FB01E40FF51FAA
:102D9000E752FE4F208130E0092E02C0369527957C
:102DA0000A94E2F721703327042E01C0220F0A94FF
:102DB000EAF7822B4F5F5F4F4530510531F7089599
:102DC000BF92CF92DF92EF92FF920F931F93CF9318
:102DD000DF938C01C0900102D0900202E0900302C8
:102DE000F09004028091050290910602A0910702E2
:102DF000B0910802C82AD92AEA2AFB2ACFE1D0E0FA
:102E0000D701C6010C2E04C0B695A7959795879556
:102E10000A94D2F780FD04C0219790F7B12C07C027
:102E2000BC2EB8018C2F0E940D070197A9F38B2DA2
:102E3000DF91CF911F910F91FF90EF90DF90CF9096
:102E4000BF900895CF93DF93EC010E94E016BE017E
:102E50000E940D07DF91CF9108951F93CF93DF93C9
:102E6000EB019091A001992321F0CB010E94221740
:102E700013C0882349F0CB010E94E016182F682F59
:102E8000CE010E94891604C0CB010E94B416182FEF
:102E9000BE01812F0E940D07DF91CF911F910895F0
:102EA00080910902859585958595089580910902FF
:102EB0008770089590910902977081E009F480E08D
:102EC000089580912D02089590912D02892B809371
:102ED0002D020895809590912D02892380932D02D3
:102EE000089510922D02089590912C02892B8093C1
:102EF0002C020895809590912C02892380932C02B6
:102F0000089510922C02089590912B02892B8093A2
:102F10002B020895809590912B02892380932B0298
:102F2000089510922B02089580910A020895089541
:102F30000C9497170C94981790910A02981721F007
:102F400080930A020C949A17089580910A028823AC
:102F500029F010920A0280E00C949A170895E091EB
:102F60000001F091010180912D028083E091000128
:102F7000F0910101908180912C02892B8083E09156
:102F80000001F0910101908180912B02892B8083B7
:102F900080910A02882381F0E0910001F091010103
:102FA0009081892B808380910001909101010E9482
:102FB000C31881110E94A517809100019091010111
:102FC0000C944F0C0C94971798E0899F9001112452
:102FD000262B209309020E94EB158091090285950A
:102FE000859585950C94E2171092090280E00C9467
:102FF000E217209109028095822380930902982F7D
:10300000977079F430E0482F082E000C550B2417E8
:10301000350739F08595859585950E940C160C9499
:10302000F417089580E090E00E94CE2521E08C3EC8
:103030009E4F09F020E0822F089582E090E00C94EA
:10304000C625682F82E090E00C94D42583E090E0C0
:103050000C94C625682F83E090E00C94D425CF9380
:1030600084E090E00E94C625C82F81E290E00E9493
:10307000C6252C2F30E0A901582BCA01CF91089505
:10308000CF93C92F682F84E090E00E94D4256C2F45
:1030900081E290E0CF910C94D425AB01BC018FE08C
:1030A00090E00C94E625AB01BC0183E190E00C9428
:1030B000E62560E070E0CB010C94531860E070E00E
:1030C000CB010E944D180C9459186CEE7EEF80E0F5
:1030D00090E00E94F22560E082E090E00E94D4251A
:1030E00060E083E090E00E94D425109205021092E7
:1030F0000602109207021092080260E084E090E05D
:103100000E94D42560E081E290E00E94D42560E036
:1031100085E090E00E94D42560E086E090E00E9487
:10312000D4256FEF87E090E00E94D42540E050E086
:10313000BA0188E090E00E94E62560E08DE090E032
:103140000E94D42540E050E0BA0188E190E00E945E
:10315000E62560E087E190E00E94D42540E050E061
:10316000BA018CE190E00E94E62560E080E290E008
:103170000E94D4250C945E180C946518682F8EE07C
:1031800090E00C94D425FC013296809114018823A0
:1031900031F080917B0287FF02C09EE101C096E082
:1031A00080E0915028F021912223D9F38F5FF9CF4D
:1031B0000895662351F1209114012223E9F0209112
:1031C0007B0227FF19C0462F4695469546954E31FE
:1031D000E0F4677021E030E002C0220F331F6A95EF
:1031E000E2F7FC01E40FF11D828190E028233923EE
:1031F00081E0232B69F409C0FC01329608962191E5
:10320000621729F0E817F907D1F780E0089581E007
:1032100008959C01FC0132969FEF80E04191461792
:1032200089F09F3F19F4411101C0982F8F5F8630BC
:10323000A9F79F3F39F0F901E90FF11D97FDFA95C4
:103240006283089508959C012A5F3F4FFC014281EB
:10325000461301C01282019682179307B9F70895A9
:10326000262F2695269526952E3168F4FC01E20F2F
:10327000F11D677021E030E001C0220F6A95EAF786
:103280008281282B22830895262F26952695269520
:103290002E3170F4FC01E20FF11D677021E030E087
:1032A00001C0220F6A95EAF72095828128232283A4
:1032B000089520911401222329F020917B0227FDFB
:1032C0000C9430190C94091920911401222329F02F
:1032D00020917B0227FD0C9444190C942319209112
:1032E0001401FC013296222331F080917B0287FF8A
:1032F00002C08EE101C086E0DF011D928A95E9F7E8
:10330000089508950C9481190C948119CF930E940B
:1033100084190E9465090E948219C0E08C2F0E94C6
:10332000FC08892B29F4CF5FC530C1F780E001C0CC
:1033300081E0CF9108950C9481190C949B190E94FF
:103340009D1980918102843049F110922F0220E46E
:1033500088E190E00FB6F894A895809360000FBEC6
:103360002093600080E00E9498060E949D1983B718
:10337000817F846083BF83B7816083BF78948895A1
:1033800083B78E7F83BF0FB6F894A89580916000B5
:10339000886180936000109260000FBE08950C94C5
:1033A00081190E9495110E94430C0E9498060C946A
:1033B000CF191F920F920FB60F9211248F939F93E4
:1033C000AF93BF9380912F02811113C08091770238
:1033D00090917802A0917902B0917A024196A11D54
:1033E000B11D8093770290937802A0937902B093F5
:1033F0007A02BF91AF919F918F910F900FBE0F9066
:103400001F90189582E084BD93E095BD9AEF97BD1B
:1034100080936E0008952FB7F89480917702909171
:103420007802A0917902B0917A022FBF08959C0191
:103430004FB7F8948091770290917802A091790229
:10344000B0917A024FBF821B930B089578941F921C
:103450000F920FB60F9211248F939F93AF93BF9348
:103460008091770290917802A0917902B0917A02CE
:103470000196A11DB11D8093770290937802A093CD
:103480007902B0937A02BF91AF919F918F910F9083
:103490000FBE0F901F90189581E08093E00080E2AE
:1034A0008093D8001092C9008FE19EE40197F1F754
:1034B00000C0000087E090EBDC0180938A029093CB
:1034C0008B02A0938C02B0938D029CE088E10FB632
:1034D000F894A895809360000FBE90936000FFCF92
:1034E000AF92BF92CF92DF92EF92FF920F931F9312
:1034F000CF93C0E0CC24C394D12CE82EF12C8C2F98
:103500000E94FC085C0100E010E0C601002E02C031
:10351000880F991F0A94E2F78A219B21892B31F4A5
:103520000F5F1F4F0C30110581F70AC0602F7C2FF1
:1035300080E00E94F206E816F90691F781E004C0E7
:10354000CF5FC530E1F680E0CF911F910F91FF90E2
:10355000EF90DF90CF90BF90AF900895CF93C82F9A
:103560008CE20E94701A882321F08C2FCF910C944A
:10357000701A80E0CF910895CF930E9412188111A4
:1035800002C00E94BC18C5E6C15049F00E946509FE
:103590008FE39CE90197F1F700C00000F5CF89E2C5
:1035A0000E94AE1A811120C18AE20E94AE1A8111D6
:1035B0000E94BC1885E00E94AE1A81110E944C1A2C
:1035C0000E941D1880932E0287E00E94AE1A882365
:1035D000A9F18BE10E94AE1A882351F080912E024E
:1035E00081FB222720F991E0922790FB81F90EC000
:1035F0008EE00E94AE1A882361F080912E0282FB39
:10360000222720F991E0922790FB82F980932E02E5
:1036100015C080E10E94AE1A90912E02882341F0DD
:1036200093FB222720F981E0822780FB93F904C0D5
:10363000892F809580FB90F990932E0280912E0225
:103640000E9421180E942F1890937C0280937B0285
:1036500080EE0E94AE1A882341F080917B02982F61
:10366000909590FB80F980937B0289E30E94AE1ACB
:10367000882359F080917B0281FB222720F991E079
:10368000922790FB81F980937B0282EE0E94AE1A12
:10369000882359F080917B0282FB222720F991E058
:1036A000922790FB82F980937B0286EE0E94AE1AED
:1036B000882359F080917B0283FB222720F991E037
:1036C000922790FB83F980937B0283EE0E94AE1ACF
:1036D000882359F080917B0284FB222720F991E016
:1036E000922790FB84F980937B0285E30E94AE1AB7
:1036F000882359F080917B0285FB222720F991E0F5
:10370000922790FB85F980937B0281E30E94AE1A99
:10371000882359F080917B0286FB222720F991E0D3
:10372000922790FB86F980937B0281E10E94AE1A7A
:10373000882359F080917B0287FB222720F991E0B2
:10374000922790FB87F980937B0280917B02909176
:103750007C020E94401887E20E94AE1AC82F8EE1B8
:103760000E94AE1A8111C2608FE10E94AE1A8111CF
:10377000C46080E20E94AE1A8111C86081E20E949A
:10378000AE1A8111C06182E20E94AE1A8111C0623C
:1037900083E20E94AE1A8111C06484E20E94AE1AD4
:1037A000882311F0C06802C0CC2329F08C2F0E941E
:1037B0002A186C2F03C00E942618682F70E080E042
:1037C00090E00E948B158FE00E94AE1A882319F0BA
:1037D00081E00E94BE1885E10E94AE1A882321F084
:1037E00080E0CF910C94BE18CF910895809137025C
:1037F00080FF0BC06091070185E0689FB001112434
:1038000075956795759567952BC081FF09C0609187
:10381000070185E0689FB00111247595679520C068
:1038200082FF07C06091070185E0689FB001112405
:1038300017C0909136029923D1F060910601961736
:1038400088F72091070185E0289F90011124929F1D
:10385000A001939F500D112470E0CA010E94982589
:103860006038710540F46115710519F406C065E012
:1038700070E0862F08958FE7089581E00895809184
:10388000370280FF08C06091030170E0759567956D
:103890007595679521C081FF06C06091030170E0B6
:1038A0007595679519C082FF04C06091030170E0AF
:1038B00010C090913602992399F0609102019617F9
:1038C000A0F780910301899FC001112470E00E943C
:1038D00098256038710540F46115710519F406C02A
:1038E00061E070E0862F08958FE7089581E00895E4
:1038F000803F21F40E94F61B819504C0813F29F48A
:103900000E94F61B80933B020895823F21F40E949F
:10391000F61B819504C0833F29F40E94F61B809317
:103920003A020895893F19F40E943F1C05C08A3F5E
:1039300031F40E943F1C819580933C0208958B3F97
:1039400021F40E943F1C819504C08C3F29F40E9401
:103950003F1C80933D020895843F21F480913902F9
:10396000816017C0853F21F480913902826011C0C7
:10397000863F21F48091390284600BC0873F21F497
:1039800080913902886005C0883F31F48091390206
:1039900080618093390208958D3F21F48091370230
:1039A00081600BC08E3F21F480913702826005C098
:1039B0008F3F29F480913702846080933702089505
:1039C000803F39F480913B0287FF6CC010923B022C
:1039D00069C0813F29F480913B021816BCF362C094
:1039E00090913A02823F29F497FF5CC010923A020C
:1039F00059C0833F19F41916CCF354C0893F41F4E0
:103A000080913C0218160CF04DC010923C024AC046
:103A10008A3F29F480913C0287FF44C0F6CF8B3F58
:103A200039F480913D0287FF3DC010923D023AC0BB
:103A30008C3F29F480913D021816BCF333C0843FBB
:103A400021F4809139028E7F17C0853F21F4809147
:103A500039028D7F11C0863F21F4809139028B7F1E
:103A60000BC0873F21F480913902877F05C0883FD2
:103A700031F4809139028F7E8093390213C08D3FDB
:103A800021F4809137028E7F0BC08E3F21F480910C
:103A900037028D7F05C08F3F29F4809137028B7FDD
:103AA0008093370280913A0281110EC080913B02CF
:103AB00081110AC080913C02811106C080913D02B3
:103AC000811102C010923602089588E392E00E94AC
:103AD000690C0E940B1A909335028093340208956A
:103AE000CF93DF9300D000D000D0CDB7DEB786E013
:103AF000E8E3F2E0DE01119601900D928A95E1F77C
:103B000080913A02811105C080913B02882309F41B
:103B10007AC080913202909133020E94171AAC0150
:103B200090913602992339F02091080130E0241752
:103B3000350758F068C0209109018AE0289F90015C
:103B400011242417350718F05EC09F3F19F09F5FBE
:103B50009093360210923C0210923D0280913A02FC
:103B6000181624F40E94F61B80933A0280913A02C0
:103B700087FF05C00E94F61B819580933A028091D1
:103B80003B02181624F40E94F61B80933B0280919E
:103B90003B0287FF05C00E94F61B819580933B0284
:103BA00030913A023323E1F020913B022223C1F00D
:103BB00045EB3403C0011124992319F090933A0284
:103BC00003C081E080933A0235EB2303C001112446
:103BD000992319F090933B0203C081E080933B024C
:103BE0000E94651D809134029091350290933302BA
:103BF0008093320286E0FE013196A8E3B2E00190A4
:103C00000D928A95E1F780913C02811105C0809167
:103C10003D02882309F47AC08091300290913102EC
:103C20000E94171AAC0190913602992339F0209125
:103C3000040130E02417350758F068C020910501D1
:103C40008AE0289F900111242417350718F05EC0E0
:103C50009F3F19F09F5F9093360210923A021092A4
:103C60003B0280913C02181624F40E943F1C809372
:103C70003C0280913C0287FF05C00E943F1C819559
:103C800080933C0280913D02181624F40E943F1C50
:103C900080933D0280913D0287FF05C00E943F1C3A
:103CA000819580933D0230913C023323E1F02091D5
:103CB0003D022223C1F045EB3403C00111249923B6
:103CC00019F090933C0203C081E080933C0235EBF5
:103CD0002303C0011124992319F090933D0203C0DE
:103CE00081E080933D020E94651D80913402909195
:103CF0003502909331028093300286E0FE013196C6
:103D0000A8E3B2E001900D928A95E1F726960FB6EE
:103D1000F894DEBF0FBECDBFDF91CF910895E8E3E9
:103D2000F2E086E0DF011D928A95E9F710923602F3
:103D300010923702089580915E020895CF93DF9329
:103D400000D01F92CDB7DEB790918102943019F563
:103D500089837B836A8382E08093E9008FEF90916F
:103D6000E800815095FD06C095ED9A95F1F70000A9
:103D70008111F5CF8091E80085FF0DC040E050E053
:103D800063E070E0CE0101960E94FA208091E80085
:103D90008E778093E8000F900F900F90DF91CF9176
:103DA0000895CF93DF93EC010E94DD20823011F063
:103DB000843031F4BE0184E0DF91CF910C949E1EDB
:103DC000DF91CF910895BC0183E00C949E1ECF93A8
:103DD000DF93EC010E94DD20823011F08430F9F491
:103DE00082E08093E9008FEF9091E800815095FD8B
:103DF00006C095ED9A95F1F700008111F5CF8091FD
:103E0000E80085FF0CC040E050E066E070E0CE01C5
:103E10000E94FA208091E8008E778093E800DF917D
:103E2000CF910895CF93DF93EC010E94DD20823083
:103E300011F08430D9F580911401882339F08091F4
:103E40007B0287FF03C060E282E002C068E081E09D
:103E50008093E9008FEF9091E800815095FD06C0B6
:103E600095ED9A95F1F700008111F5CF8091E8006A
:103E700085FF1CC080911401811105C040E050E015
